:100000000200B8028003FFFFFFFFFF02800BFFFF2B
:10001000FFFFFF028013FFFFFFFFFF02801BFFFFB8
:10002000FFFFFF028023FFFFFFFFFF02802BFFFF88
:10003000FFFFFF020AA5020A5702168DFFFFFFFF0E
:100040000229B90229CE0229D70229E40229EC02A9
:100050002A06022A10022A1B022A27022A56022AEC
:1000600092022AB2022ABF022ACC022AD3022ADA38
:10007000022AEA022AFC022B0E022B20022B2F025C
:100080002B3C022B4B022B5A022B67022B79022BA3
:100090008A022B9D022BA8022BBD022BC5022BD658
:1000A000022BDE022BF1022BFC022C2D022C4A0229
:1000B0002C60022C7F022CA97A407B00DBFEDAFA4E
:1000C00075819DE556B4A5030201A478087AF876F7
:1000D0000008DAFB758920759852758DFDD28E90D7
:1000E0000000209825000000A3E583458270F3906E
:1000F0008000E0B400030200DFB4FF030200DF75FC
:100100005280755300C053C05222122BD6B4F00057
:10011000400C7A198587F0D2F785F0878029B420C2
:10012000047A968022B400E2122BD6B40007758DB3
:10013000E87A128012B48007758DF47A248008B4AE
:10014000F8C8758DFA7A488A577A16122BC5DAFBE9
:100150009001C3122BA89001DD122BA89001F91277
:100160002BA8E557C0E0122B8AD0E0B419057432F1
:10017000122B79E4122B8A122BC5900216122BA88F
:10018000120221E55C122B8AE55D122B8A122BC527
:10019000122BC57556A5754E80754F00755080752C
:1001A00051008019758920759852E557122BFCD2A1
:1001B0008E122BC5122BC5900205122BA8120A8293
:1001C00002112452454D35352052656D6F746520FE
:1001D0004D6F6E69746F722076332E300D32303071
:1001E000352053696C6120526573656172636820C4
:1001F000436F2E2C4C74642E0D4261756420526145
:100200007465203A0053797374656D205265736587
:1002100074202E2E2E0D436865636B73756D203A26
:10022000007583007582007A2C7BB8755C00755D63
:1002300000E493121B9A122A9270F62275819D7423
:100240002D122B79121E4C900070121DA5BD0003BB
:1002500002023CBD010302025C020299C083C0821B
:10026000122A061229B1F5F07B009002DAE4930B12
:10027000A3B40007D082D083020299B5F0EF9002B8
:10028000F18002A3A3DBFCE493FA740193FBD08218
:10029000D083EBC0E0EAC0E02275819D7A007B70DC
:1002A000122A92600A122A061229B1B420F2A3750A
:1002B000819DAA83AB82900070122BD0122A92A348
:1002C00070F79002CB122BA802023C5E2053796E8D
:1002D000746178204572726F720D41424344454605
:1002E0004748494C4D4E4F5051525354555658590A
:1002F00000031D078607A80880094209A209E90B27
:10030000130E990FC510C411061BA611421230120C
:100310006215A1162917381A7F1B501D03121E2CB7
:10032000BD00030202AF8A608B61121E42856083AA
:10033000856182122B9D743A122B79121E4C120782
:1003400072900070121D86BD000302023C12035819
:10035000B400DA12049780D5E4F55AF55BF55CF544
:100360005DF55EF55FC083C0827A04900099122922
:10037000A9A3DAFAD082D083858362858263BD091E
:1003800000400302046F12075D121F35B400030220
:10039000046F9000991229A9856283856382121DDA
:1003A00086BD000302046D858362858263BD0900FA
:1003B000400302046F12075D12204CB400030203D5
:1003C000C990009A1229A980131206BFB400030233
:1003D000046F90009A1229A98A5A8B5B85628385E3
:1003E0006382121D86BD000302046D8583628582CF
:1003F00063BD0900400302046F12075D12204CB474
:10040000000302040D90009B1229A980131206BF5D
:10041000B4000302046F90009B1229A98A5C8B5DD3
:10042000856283856382121D86BD000302046D858B
:100430008362858263BD0900503512075D12204C2E
:10044000B4000302044E90009C1229A980131206E6
:10045000BFB4000302046F90009C1229A98A5E8B2E
:100460005F856283856382121D86BD0002E422904F
:100470000478122BA87401222020202020417373BD
:10048000656D626C65722053796E74617820457277
:10049000726F722021070D90009978667A041229F4
:1004A000B1F6A308DAF89024A97F007A047B0078DB
:1004B00066EB93F5F0E6B5F006080BDAF4800E7AF9
:1004C000007B05122A100FBF00E10205568F6674EB
:1004D0000493C0E0540FF569D0E0C4540FB4012D6B
:1004E000E55A54F8F5F0E56054F8B5F069E55AC4FA
:1004F0002354E0F5F0E493B40106E5F044118004E0
:10050000E5F04401F566E55BF567020637B4020BDA
:10051000E55AF567E55BF568020637B4031E74011A
:1005200093B4010CE55AB4002DE55BF5670206377C
:10053000E55CB40021E55DF567020637B4041AE511
:100540005AB40012E55BF567855C83855D8212060F
:1005500075F56802063702064EB4051E740193B4A1
:10056000010CE55AB400EFE55BF567020637E55C80
:10057000B400E3E55DF567020637B40615E55AB445
:1005800000D4E55BF568E55CB400CBE55DF567029A
:100590000637B40715E55AB400BCE55BF567E55CC2
:1005A000B400B3E55DF568020637B408347401930E
:1005B000B40117E55AB4009EE55BF567855C838559
:1005C0005D82120675F568020637E55CB40087E5C2
:1005D0005DF567855E83855F82120675F5680206A4
:1005E00037B4090CE55CB40065E55DF567020637D4
:1005F000B40A16E55CB40056E55DF567855E838553
:100600005F82120675F568802EB40B0AE55CF5670B
:10061000E55DF5688021B40C1E740193B4010D856D
:100620005A83855B82120675F567800B855C83852E
:100630005D82120675F5678560838561827866AF95
:1006400069E6F0A308DFFA8583608582612290065F
:1006500055122BA8222020202020417373656D6243
:100660006C657220436F6D6D616E64204572726FB0
:10067000722021070DAA60AB61E569142BFB7400A1
:100680003AFA122A9260154013122A1B122A06E522
:1006900083B40023E582B48000501C22C583CAC500
:1006A00083C582CBC582122A1BE583B40009E5828B
:1006B000B480005002F42212064ED0E0D0E022E5D1
:1006C00066B423047F02800BB42F047F0380047F71
:1006D00001800F786679677A07E7F60809DAFA7514
:1006E0006D20E566B43000404CB43A00504778665F
:1006F0007A007B007C007D08E6B4300508DDF980D7
:100700002BE6B4200302072CB4480302072CB430B4
:10071000004020B44700501BB441005005B43A00DB
:100720005011122C56121E11080CDDD5BC050050BC
:1007300002EF22E422122102B400030207437A00EE
:10074000FBEF22122205B400030207517A00FBEFEF
:1007500022E42278667A08762008DAFB2212075310
:10076000ED7A00FB122A1B78661229B1F608A3DD88
:10077000F8229000707A281229B1B42C0574201246
:1007800029A9A3DAF222121E2CBD00030207998ABE
:10079000548B55121E4202023C85548385558212A9
:1007A0002B9D122BC502023C121E2CBD000302021F
:1007B000AF8A608B61121E2CBD00030202AF8A62F9
:1007C0008B63121DA5BD00030202AFBC006BBD050B
:1007D0000040030202998A648B65121E4285608381
:1007E000856182AC64AD65E0F5F0C083C0828C8326
:1007F0008D82E0D082D083B5F01574012DFD740098
:100800003CFCAA62AB63122A92A370DB02023CFF9B
:10081000122B9D743A122B79E5F0122B8A122BD0F1
:10082000EC122B8AED122B8A743A122B79EF122BD1
:100830008A122BC580C4020299BD01FA122A06123F
:1008400029B1A3B448F0121E2CBD0003020299BACC
:1008500000E48B5A121E42856083856182E0B55A9E
:100860000DAA62AB63122A92A370F202023CFF123D
:100870002B9D743A122B79EF122B8A122BC580E133
:10088000121E2CBD00030208A38A508B51121E2C8D
:10089000BD00030208B98A628B63121E421208CFA0
:1008A00002023CAA50AB5190007F122A108583624D
:1008B0008582631208CF02023CAA50AB5190007FA0
:1008C000122A108583628582631208CF02023CE5FA
:1008D00050122B8AE551122B8A743A122B79122B63
:1008E000D07E08855083855182122AD3E0A3122B33
:1008F0008A122BD0DEF6742D122B79122BD07E08A3
:10090000E0A3122B8A122BD0DEF6122BD0122BD0A2
:100910008583508582517E10122ACCE0A3B47F00DB
:100920005005B420005007742E122B798003122B2F
:1009300079DEE8122BC5AA62AB63122A926090405E
:100940008E22121E2CBD00030202AF8A608B611240
:100950001E42856083856182122B9D743A122B7929
:10096000E0122B8A122BD0121E4C900070121DA583
:10097000BD000302023CBC010302099ABA001BEB52
:10098000C0E0121DA5D0E0BD0010856083856182A6
:10099000F0A385836085826180B87407122B790289
:1009A0000952121E2CBD00030202AF8A608B611235
:1009B0001E2CBD00030202AF8A628B63121E2CBD87
:1009C00000030202AFBA001E8B5A121DA5BD00160D
:1009D000856083856182AA62AB63E55AF0122A9230
:1009E000A340F702023C020299121E2CBD00030232
:1009F00009F98A528B53121E42855283855382E431
:100A000093B40009900A49122BA802023C756900B0
:100A1000E55445556028855483855582AA52AB53C9
:100A2000122A9260194017E0F5667402F0A3E0F50F
:100A3000677400F0A3E0F5687436F0756901120A76
:100A4000CA854881C053C052224E6F2050726F67D2
:100A500072616D2021070D85814875819D120AF014
:100A6000855452855553120A8285528385538212CA
:100A70002B9D900A7B122BA802023C2042726561DA
:100A80006B0DE569B4000122B401128554838555CC
:100A900082E566F0A3E567F0A3E568F0228564834C
:100AA00085658280EC85814875819D120AF0120A65
:100AB00082900ABA122BA802023C456E6420507242
:100AC0006F6772616D202E2E2E0DE54B5418B40009
:100AD00010A840A941AA42AB43AC44AD45AE46AFD5
:100AE00047854982854A83854BD0E54C854DF02268
:100AF00085824985834A85D04BF54C85F04DC2D31C
:100B0000C2D4884089418A428B438C448D458E46AD
:100B10008F4722121E42900B32E493A3B4000302CB
:100B2000023CB40D03020B2D122B7980EC122BC565
:100B300080E752454D353520436F6D6D616E642001
:100B400053756D6D617279202E2E2E0D41206164DA
:100B5000647220202020202020202020202041738B
:100B600073656D626C65720D42205B616464725DD9
:100B700020202020202020202020427265616B2030
:100B80005365742F446973706C61790D43207261F1
:100B90006E67652061646472202020202020436FEE
:100BA0006D7061726520426C6F636B0D2020726105
:100BB0006E67652048206279746520202020436F8D
:100BC0006D7061726520427974650D44205B6164CB
:100BD00064725D205B616464725D202020446973EF
:100BE000706C6179204D656D6F72790D452061647F
:100BF0006472202020202020202020202020456EEC
:100C000074657220446174610D462072616E67657F
:100C1000206279746520202020202046696C6C2099
:100C20004D656D6F72790D47205B616464725D2064
:100C3000202020202020202020476F202852756E61
:100C4000290D482020202020202020202020202086
:100C50002020202048656C700D49205B616464721F
:100C60005D20202020202020202020496E746572E5
:100C70006E616C2052414D205365742F446973702E
:100C80006C61790D4C205B616464725D20202020D2
:100C9000202020202020646F776E4C6F61642049F3
:100CA0004E54454C2D4845582046696C6520667267
:100CB0006F6D2050430D4D2072616E676520616439
:100CC00064722020202020204D6F7665204D6F6DAE
:100CD0006F72790D4E2020202020202020202020FF
:100CE0002020202020204E65772028436C656172EB
:100CF000205573657220494E542D52414D2C20527F
:100D000065676973746572202620534652290D4F1A
:100D1000206269742D706F7274205B302C315D20FD
:100D2000204F757420506F72740D502072616E6781
:100D300065202020202020202020202075506C6F4E
:100D4000616420494E54454C2D4845582046696CF5
:100D50006520746F2050430D51202020202020203A
:100D60002020202020202020202051756974202858
:100D7000506F776572206F6666206F7220526573C0
:100D80006574290D52205B7265672076616C75650C
:100D90005D202020202052656769737465722026CB
:100DA00020534652205365742F446973706C6179E7
:100DB0000D532072616E67652062797465202E2E56
:100DC0002E2020536561726368204D656D6F7279C6
:100DD0002028382042797465204D6178290D5420EF
:100DE0005B616464725D2020202020202020202070
:100DF0005472616365202853696E676C6520537473
:100E00006570290D55205B616464725D205B6164CF
:100E100064725D202020556E617373656D626C6530
:100E200072202850726F6772616D204D656D6F7210
:100E300079290D562020202020202020202020202D
:100E40002020202020566563746F722041646472F4
:100E500065737320496E746572727570740D5820D5
:100E600072616E6765202020202020202020202015
:100E700046696E6420436865636B73756D0D592018
:100E8000706F72742020202020202020202020201D
:100E9000496E20506F72740D00121E2CBD000302AB
:100EA0000EA5020F6A7F00EF122B8A743A122B797B
:100EB000122BD07E08EFFDED120F550D122B8A126A
:100EC0002BD0DEF3742D122B79122BD07E08ED126D
:100ED0000F550D122B8A122BD0DEF3BF4002801C5F
:100EE000BF50028017BF60028012BF7002800DBF2A
:100EF00080028008BF90028003BFA007742A122BD3
:100F0000798003122BD0122BD07E10EF120F550FC9
:100F1000B47F005005B420005007742E122B798046
:100F200003122B79DEE5122BC5BF0009900F381292
:100F30002BA802023C020EA728202A203D204D6F3C
:100F40006E69746F7220576F726B696E67204172A1
:100F5000656120290DB4080050022440F8E622B44F
:100F6000080050022440F8EAF622BA0003020F7388
:100F70000202998B60121E42E560122B8A743A12AB
:100F80002B79E560120F55122B8A122BD0121E4CB2
:100F9000900070121DA5BD000302023CBC010302BB
:100FA0000FBDBA0018EBC0E0121DA5D0E0BD000DCA
:100FB000FAE560120F5FE56004F56080BB7407120C
:100FC0002B79020F78121E2CBD0003020FD98A6004
:100FD0008B617E01121E4280087560007561007E83
:100FE00000901096122BA8122BD6B40D03020FE717
:100FF000B40A03020FE7B44F03021083B453030291
:101000001081B43A03021011021078122BD6B43AB0
:10101000FA7F00122BEAFD122BEAF583122BEAF578
:1010200082122BEAB4003DBE0119AA83AB8285600F
:1010300083856182122A1B8583608582618A838B06
:10104000827E00AA60AB61122A10122BEAF0A3DDA7
:10105000F9EFF404F5F0122BEAB5F01C122BD612BE
:101060002BD680A7EFF404F5F0122BDEB5F00912B1
:101070002BD6122BD602023C9010B2122BA80202E1
:101080003C7E01122BDEF560122BDEF561122BD6B1
:10109000122BD6020FE7446F776E6C6F61642049A4
:1010A0004E54454C2D4845582046696C65202E2EDF
:1010B0002E0D446F776E6C6F6164204552524F5213
:1010C0002021070D121E2CBD00030202AF8A608B87
:1010D00061121E2CBD00030202AF8A628B63121ED6
:1010E0002CBD00030202AF8A648B65121DA5BD00F2
:1010F00012AA60AB61AC62AD63AE64AF65121EB89C
:1011000002023C020299121E4278087A38760008E0
:10111000DAFB78B07A50760008DAFB78407A087605
:101120000008DAFB754C00754D00754B00754807DB
:10113000754A007549007590FF755280755300021D
:10114000023C121E2CBD00030202AF8A608B6112AA
:101150001E2CBD00030202AF8A628B63121E4290F6
:1011600011F7122BA8901211122BA8122BD6B40D26
:10117000FA8560838561827D007F00743A122B7945
:101180001211B7EE122B96E583122B96E582122BE5
:1011900096E4122B96E0122B96A3DEF9EFF40412DC
:1011A0002B8A122BC5BD01D19011EB122BA8122B4B
:1011B000D6B40DFA02023CE583CAF583E582CBF58D
:1011C00082856283856382122A1BE5837016E5821D
:1011D000B40F030211E2500C7D01AE820E8A838BA4
:1011E00082227D018A838B827E10223A3030303019
:1011F0003030303146460D55706C6F616420494E79
:1012000054454C2D4845582046696C65202E2E2E9D
:101210000D5479706520454E54455220746F20530B
:101220007461727420616E642046696E6973680D22
:10123000121E4290123E122BA875560080FE524597
:101240004D35352051554954202120506F77657216
:10125000206F6666206F72205265736574202E2E93
:101260002E0D121DA5BD000302126E0214A69013CE
:101270005A122BA8E54B03030354034430122B7975
:10128000122BC5901369122BA8E54B0303035403DB
:1012900075F008A47F08C0E0120F55122B8A122B9C
:1012A000D0D0E004DFF0B40805742A122B79122B99
:1012B000C5901381122BA89013CD122BA8E54812CC
:1012C0001484122BA8E549121484122BA8E54A12A3
:1012D0001484122BC5122BA8E587121496122BA882
:1012E000E588121496122BA8E589121496122BC5C4
:1012F000122BA8E590121496122BA8E598121496BA
:10130000122BA8E5A8121496122BC5122BA8E5B82B
:10131000121496122BA8E5C8121496122BA8E54BAE
:10132000121484122BC5122BA8E54C121484122B14
:10133000A8E54D121484122BC59013A2122BA812EB
:101340002BD0855283855382122B9D122BD0122BCA
:10135000D09013B4122BA802023C526567697374D3
:1013600065722042616E6B20005230205231205253
:1013700032205233205234205235205236205237F8
:101380000D5370656369616C2046756E6374696F97
:101390006E205265676973746572732028534652D4
:1013A000290D50726F6772616D20436F756E7465A1
:1013B00072203D0028202A203D20566972747561F4
:1013C0006C20526567697374657220290D20202096
:1013D000535000202044504C00202044504800200E
:1013E00050434F4E002054434F4E0020544D4F4425
:1013F000002020205031002053434F4E0020202059
:101400004945002020204950005432434F4E0020CF
:1014100020505357002020414343002020202042E9
:101420000020202052300020202052310020202097
:10143000523200202020523300202020523400203D
:101440002020523500202020523600202020523704
:1014500000F55A743D122B79E55A122B8A122BD0C3
:10146000743C122B79E55A7F0833C0E04007743092
:10147000122B7980057431122B79D0E0DFEB743EAA
:10148000122B7922121451122BD0742A122B79129A
:101490002BD0122BD022121451122BD0122BD0127F
:1014A0002BD0122BD022BD06004003020299858367
:1014B00062858263786A122A061229B1F618DDF66F
:1014C000B86600400576201880F67A137BCD7E0141
:1014D0008A838B8278667F05E6F55AE493B55A06CF
:1014E00008A3DFF480190EBE170985628385638225
:1014F000020299900006122A10AA83AB8280D18E34
:101500005A856283856382121E2CBD00030202AFDE
:10151000BA00030215190202998B5B121E42AB5BE3
:10152000E55AB401048B488072B402048B49806B85
:10153000B403048B4A8064B404048B87805DB405D3
:10154000048B888056B406048B89804FB407048BC3
:10155000908048B408048B988041B409048BA8801B
:101560003AB40A048BB88033B40B048BC8802CB413
:101570000C048B4B8025B40D048B4C801EB40E04E0
:101580008B4D8017C3940FFAE54B03030354037587
:10159000F008A42A8BF0AAF0120F5F02023C0202AC
:1015A00099121E2CBD00030202AF8A608B61121ECD
:1015B0002CBD00030202AF8A628B63121E2CBD0099
:1015C000030202AFBA00D78B6678677A0876000804
:1015D000DAFB755A67121E2CBD00030215F0A85ADB
:1015E000B86E03020299BA00B5EBF608885A80E596
:1015F000856083856182C083C0827866E0C396700F
:1016000011A308B600F6856083856182122B9D12B6
:101610002BC5D082D083AA62AB63122A92A38583A2
:101620006085826170D002023C121E2CBD00030254
:1016300016398A528B53121E42855283855382E497
:1016400093758300F5827A007B05122A277A247B22
:10165000A9122A10740493540F7A00FB85528385D3
:101660005382122A10858364858265E0F5667402D0
:10167000F0A3E0F5677400F0A3E0F5687439F07545
:101680006902120ACA854881C053C0522285814826
:1016900075819D120AF0856452856553120A829005
:1016A0001712122BA8855283855382122B9D9017F7
:1016B00016122BA8E54C122B8A90171A122BA8E5AC
:1016C0004D122B8A90171E122BA8854A83854982BA
:1016D000122B9D901725122BA8E54B122B8A9017E1
:1016E0002B122BA8E548122B8A901730122BA8E555
:1016F0004B030303540375F008A47F08C0E0120FE6
:1017000055122B8A122BD0D0E004DFF0122BC50229
:10171000023C50433D0020413D0020423D0020441A
:101720005054523D00205053573D002053503D002F
:101730002052302D52373D00121E2CBD0009756419
:101740000112176A02023C8A4E8B4F121E2CBD00FA
:101750000975640112176A02023C8A628B63121EC9
:101760004275640012176A02023C756500854E835B
:10177000854F82E493758300F5827A007B05122AF7
:10178000277A247BA9122A1085835A85825BE54E2D
:10179000122B8AE54F122B8A743A122B79122BD016
:1017A000855A83855B82740493540FB40003021935
:1017B000ACFF7E0A854E83854F82E493122B8AA369
:1017C0001E1EDFF6122BD0DEFB855A83855B82E47A
:1017D00093121F267F05E493122B79A3DFF8122BB7
:1017E000D0122BD0855A83855B82740193B4000399
:1017F000021970B40103021802122035121A3C02B9
:101800001865740493C4540F854E83854F82B401C8
:1018100017E58354F8FAE493C40354074AFA7401B1
:1018200093FB1219C6021865B4020E740193FA7480
:101830000293FB1219C6021865B40C0974019312C5
:101840001A4B021865B4030302184EB4040974015C
:1018500093121A1E021865E4937A01B485027A0283
:10186000EA93121A00855A83855B82740293B4004E
:1018700003021970C0E0742C122B79D0E0B401037C
:10188000021898B40203021898B4030302189812BD
:101890002035121A3C02193DFF740493C4540F857D
:1018A0004E83854F82B40311BF0305742F122B7929
:1018B000740193121A1E02193DB4040974029312A2
:1018C0001A4B02193DB40509740193121A0002194A
:1018D0003DB40611E4937A02B485027A01EA9312C8
:1018E0001A0002193DB4070E7423122B7974029367
:1018F0001219E602193DB40817E493B4B50974014E
:1019000093121A0002193D740293121A4B02193DE8
:10191000B40B137423122B79740193FA740293FBA2
:101920001219C602193DB40C09740193121A4B0224
:10193000193D7423122B797401931219E6855A8389
:10194000855B82740393B40003021970C0E0742CA9
:10195000122B79D0E0B40103021964122035121A57
:101960003C021970854E83854F82740293121A4B84
:10197000122BC5855A83855B82740493540F7A00B9
:10198000FB854E83854F82122A1085834E85824FB8
:10199000E564B401080565E565B4100D22AA62ABE3
:1019A00063122A92600340012202176D9019B3124C
:1019B0002BA82255617373656D626C657220455268
:1019C000524F5220210DEAC4540FB40A004005744E
:1019D00030122B79EBC0E0EA122B8AD0E0122B8A6E
:1019E0007448122B7922C0E0C4540FB40A00400599
:1019F0007430122B79D0E0122B8A7448122B792282
:101A0000FE1220E7B40003021A197F06E493B42003
:101A10000122122B79A3DFF422EE1219E622FF1223
:101A200021DEB40003021A377F05E493B4200122BB
:101A3000122B79A3DFF422EF1219E6227F07E49339
:101A4000B4200122122B79A3DFF422FF855A83856B
:101A50005B82740493540F14854E83854F827A0001
:101A6000FB122A107A00EFA2E7400704FB122A10AB
:101A70008005F4FB122A1BAA83AB821219C622121C
:101A80001E42901A9EE493A3B4000302023CB40DDC
:101A900003021A99122B7980EC122BC580E7496E4C
:101AA000746572727570747320566563746F7220FA
:101AB00041646472657373202E2E2E0D312E2049E1
:101AC0004E54302020202020202020383030334831
:101AD0000D322E205446302020202020202020208F
:101AE00038303042480D332E20494E5431202020CA
:101AF000202020202038303133480D342E20544609
:101B00003120202020202020202038303142480D54
:101B1000352E205249202B205449202020202038C7
:101B2000303233480D362E20544632202B20455873
:101B30004632202038303242480D372E20454E4460
:101B40002D564543544F52202030303333480D003A
:101B5000121E2CBD00030202998A5A8B5B121E2CA6
:101B6000BD00030202998A5C8B5D121E42855A8376
:101B7000855B82AA5CAB5D755C00755D00E0121B45
:101B80009A122A9270F7E0121B9AE55C122B8AE5F2
:101B90005D122B8A122BC502023C255DF55DE55CCA
:101BA0003400F55CA322121E2CBD00030202998BA7
:101BB0005A121E2CBD00030202998B5B121E42E5D5
:101BC0005BB400028008B401028003020299A2E023
:101BD00092F0E55AB40007A2F0928002023CB401F0
:101BE00007A2F0928102023CB40207A2F0928202A4
:101BF000023CB40307A2F0928302023CB40407A2A1
:101C0000F0928402023CB40507A2F0928502023CE5
:101C1000B40607A2F0928602023CB40707A2F09233
:101C20008702023CB41007A2F0929002023CB41169
:101C300007A2F0929102023CB41207A2F092920223
:101C4000023CB41307A2F0929302023CB41407A220
:101C5000F0929402023CB41507A2F0929502023C65
:101C6000B41607A2F0929602023CB41707A2F092B3
:101C70009702023CB42007A2F092A002023CB421D9
:101C800007A2F092A102023CB42207A2F092A202A3
:101C9000023CB42307A2F092A302023CB42407A2A0
:101CA000F092A402023CB42507A2F092A502023CE5
:101CB000B42607A2F092A602023CB42707A2F09233
:101CC000A702023CB43207A2F092B202023CB43343
:101CD00007A2F092B302023CB43407A2F092B4021D
:101CE000023CB43507A2F092B502023CB43607A21A
:101CF000F092B602023CB43707A2F092B702023C5F
:101D0000020299121E2CBD00030202998B5A121E68
:101D100042E55AB400087F00121D4202023CB401A1
:101D2000087F01121D4202023CB402087F02121D0C
:101D30004202023CB403087F03121D4202023C022D
:101D40000299BF0004E5808010BF0104E59080097E
:101D5000BF0204E5A08002E5B07D0833C0E0743125
:101D600040027430122B79D0E0DDF0740D122B7923
:101D700020980A7A007B00DBFEDAFA80C5122BD6A7
:101D8000122BC502023C7D001229B1B42003A380AE
:101D9000F71229B1B42003021DA4B40D03021DA43F
:101DA0000DA380ED227A007B007C007D007E011275
:101DB00029B1B42003A380F71229B1B42003021E75
:101DC00010B40D03021E10B43000402BB447005075
:101DD00026B441005005B43A00501CBE0108B4308E
:101DE00005A37D0180D2BE01047E007D00122C5629
:101DF000121E110DA380C17C017A007B001229B153
:101E0000B42003021E10B40D03021E100DA380EDBA
:101E100022C0E0EAC454F0FAEBC4C0E054F0FBD0B6
:101E2000E0540F4AFAD0E0540F4BFB22121DA5BD1F
:101E3000000122BD05004003020299BC0103020219
:101E40009922121DA5BD0001220202999000701274
:101E50002BD6B40D071229A9122BC522B4080302F0
:101E60001E96B42000404AB47F005045122B7912D0
:101E70002CA91229A9A37A007B99122A9240D01288
:101E80002A067408122B79122BD07408122B79743D
:101E900007122B7980B97A007B70122A9260B07495
:101EA00008122B79122BD07408122B79122A068073
:101EB0009E7407122B7980978E838F82122A92400C
:101EC0003D603B8C838D82122A1BEF2582FFEE350D
:101ED00083FE8C838D82E08E838F82F08C838D8253
:101EE000122A927001228C838D82122A06AC83AD55
:101EF000828E838F82122A06AE83AF8280D48A8339
:101F00008B82E08E838F82F08C838D82122A927076
:101F100001228A838B82A3AA83AB828E838F82A3C2
:101F2000AE83AF8280D81475F005A4901F597A0053
:101F3000FB122A1022901F597C017A057B007866DB
:101F4000EB93C3967006080BDAF6EC227A007B0559
:101F5000122A100CBC2DE3E4224143414C4C414475
:101F60004420204144444320414A4D5020414E4C9E
:101F70002020434A4E4520434C52202043504C20C1
:101F8000204441202020444543202044495620201D
:101F9000444A4E5A20494E4320204A422020204A9B
:101FA000424320204A432020204A4D5020204A4EC0
:101FB0004220204A4E4320204A4E5A20204A5A208E
:101FC00020204C43414C4C4C4A4D50204D4F562004
:101FD000204D4F5643204D4F5658204D554C2020F4
:101FE0004E4F5020204F524C2020504F5020205018
:101FF0005553482052455420205245544920524CB4
:10200000202020524C432020525220202052524364
:1020100020205345544220534A4D502053554242AC
:1020200020535741502058434820205843484420CB
:1020300058524C2020B40400500122C3940475F07F
:1020400007A49020707A00FB122A10229020707C46
:10205000047A077B007866EB93C3967006080BDA68
:10206000F6EC227A007B07122A100CBC15E3E4225E
:1020700040412B4450545240412B50432020404477
:1020800050545220204052302020202040523120F5
:1020900020202041202020202020414220202020DC
:1020A0002043202020202020445054522020205221
:1020B0003020202020205231202020202052322089
:1020C0002020202052332020202020523420202085
:1020D0002020523520202020205236202020202071
:1020E000523720202020207F1AF5F0902128E493F9
:1020F000B5F004A37401227A007B07122A10DFEEE8
:10210000E4229021297C1A7A067B007866EB93C33F
:1021100096700A080BDAF6122A06E493227A007BFC
:1021200007122A10DCE1E422805030202020208198
:102130005350202020208244504C202020834450A3
:10214000482020208750434F4E20208854434F4E34
:10215000202089544D4F4420208A544C3020202088
:102160008B544C312020208C5448302020208D541A
:102170004831202020905031202020209853434F78
:102180004E202099534255462020A0503220202036
:1021900020A8494520202020B0503320202020B8FE
:1021A000495020202020C85432434F4E20CA524369
:1021B0004150324CCB524341503248CC544C3220E7
:1021C0002020CD544832202020D0505357202020AA
:1021D000E0414343202020F0422020202020B480F2
:1021E000005002E422C39480758300F5827A007B5C
:1021F00005122A277A227B29122A10E493B420029E
:10220000E4227401229022297C807A057B00786682
:10221000EB93C3967006080BDAF6EC227A007B0586
:10222000122A100CBCF8E3E42250302E302050303B
:102230002E312050302E322050302E332050302E70
:10224000342050302E352050302E362050302E374E
:102250002049543020204945302020495431202045
:1022600049453120205452302020544630202054FB
:1022700052312020544631202050312E3020503110
:102280002E312050312E322050312E332050312E1D
:10229000342050312E352050312E362050312E37FB
:1022A000205249202020544920202052423820200A
:1022B000544238202052454E2020534D3220205386
:1022C0004D312020534D30202050322E30205032BE
:1022D0002E312050322E322050322E332050322ECA
:1022E000342050322E352050322E362050322E37A8
:1022F000204558302020455430202045583120209A
:1023000045543120204553202020455432202020A0
:10231000202020204541202020525844202054587D
:10232000442020494E543020494E5431205430200E
:102330002020543120202057522020205244202099
:102340002050583020205054302020505831202028
:10235000505431202050532020205054322020202F
:10236000202020202020202020202020202020206D
:10237000202020202020202020202020202020205D
:10238000202020202020202020202020202020204D
:10239000204350524C324354322020545232202099
:1023A0004558454E32544C434B2052434C4B2045EC
:1023B0005846322054463220205020202020202011
:1023C0002020204F562020205253302020525331BD
:1023D0002020463020202041432020204359202027
:1023E00020202020202020202020202020202020ED
:1023F00020202020202020202020202020202020DD
:102400002020202020202020204143432E30414303
:10241000432E314143432E324143432E3341434304
:102420002E344143432E354143432E364143432E00
:102430003720202020202020202020202020202085
:10244000202020202020202020202020202020208C
:10245000202020202020202020422E302020422E0C
:10246000312020422E322020422E332020422E3492
:102470002020422E352020422E362020422E37208A
:10248000202020202020202020202020202020204C
:10249000202020202020202020202020202020203C
:1024A0002020202020202020201C000000010401EA
:1024B000000012170100002324090000010D09008B
:1024C00000010D010000520D070000010D08000081
:1024D000010D0D0000010D0E0000010D0F000001A7
:1024E0000D100000010D110000010D120000010D82
:1024F000130000010D140000010F01010043010150
:10250000000012160100002325090000010A09003D
:1025100000010A010000520A070000010A08000039
:10252000010A0D0000010A0E0000010A0F0000015F
:102530000A100000010A110000010A120000010A3D
:10254000130000010A140000010E01010043040100
:10255000000012200000000122090000010209020F
:102560000092020901005202090700010209080055
:102570000102090D000102090E000102090F00010C
:1025800002091000010209110001020912000102F2
:1025900009130001020914000112010100430101A5
:1025A00000001221000000012309000001030902BC
:1025B0000092030901005203090700010309080002
:1025C0000103090D000103090E000103090F0001B9
:1025D000030910000103091100010309120001039E
:1025E00009130001030914000110010000C20401D5
:1025F0000000121D010900521D010200731D090295
:1026000000921D090100521D090700011D09080063
:10261000011D090D00011D090E00011D090F00011A
:102620001D091000011D091100011D091200011DE5
:10263000091300011D0914000113010000C201016A
:10264000000012050109005205010200730509028C
:10265000009205090100520509070001050908005B
:102660000105090D000105090E000105090F000112
:1026700005091000010509110001050912000105F5
:1026800009130001050914000115010000C204012D
:102690000000122C010900522C010200732C0902C7
:1026A00000922C090100522C090700012C09080096
:1026B000012C090D00012C090E00012C090F00014D
:1026C0002C091000012C091100012C091200012C09
:1026D000091300012C0914000114010000C20101BA
:1026E0000000121D0B010032110400000118090244
:1026F00000921801020073180702009218080200E5
:1027000092180D020092180E020092180F02009209
:10271000181002009218110200921812020092186A
:1027200013020092181402009227010000C2040153
:10273000000012050B01003219090500010B0A0007
:102740000001180101006318010700521801080078
:102750005218010D005218010E005218010F0052BC
:1027600018011000521801110052180112005218DD
:10277000011300521801140052180C0200B3010199
:1027800000001218010B0032190904000128090287
:1027900000922809010052280907000128090800B1
:1027A0000128090D000128090E000128090F000168
:1027B0002809100001280911000128091200012828
:1027C0000913000128091400011D0B030032040144
:1027D000000012180B0100320D0C0000011B0A0052
:1027E0000001000000000018070100521808010055
:1027F00052180D010052180E010052180F0100521C
:10280000181001005218110100521812010052183C
:10281000130100521814010052050B03003201018C
:102820000000120801000032080B00000106090236
:1028300001A3060901018306070201A3060802019C
:10284000A3060D0201A3060E0201A3060F0201A3B7
:1028500006100201A306110201A306120201A3063B
:10286000130201A306140201A31F01000052040178
:102870000000120701000032070B000001290900C7
:1028800000012A090100522A090700012A0908004B
:10289000012A090D00012A090E00012A090F000171
:1028A0002A091000012A091100012A091200012A2F
:1028B000091300012A091400011E01000052010140
:1028C0000000122601000032260B00000109090059
:1028D00000010C010100832B090700012B090800EE
:1028E000010C0D0100C20C0E0100C20C0F0100C250
:1028F0000C100100C20C110100C20C120100C20C2C
:10290000130100C20C140100C21A090600010401DF
:102910000000121A090700011A090800010709003E
:1029200000011809010052180907000118090800E0
:102930000118090D000118090E000118090F000106
:1029400018091000011809110001180912000118D6
:102950000913000118091400011A060900010101F8
:102960000000121A070900011A08090001080900ED
:102970000001180109005218070900011808090090
:1029800001180D090001180E090001180F090001B6
:102990001810090001181109000118120900011886
:1029A000130900011814090001886FA882F6A86FA6
:1029B00022886FA882E6A86F22400820D601222430
:1029C000FAC32220D60424A0D322249AD3227BE661
:1029D0000000DBFCDAF8227BB37C00DCFE0000DBCD
:1029E000F8DAF4227A0A1229D7D9F922C083C082F0
:1029F000758300F582EA7A00FB122A27D0E0FBD02B
:102A0000E0FA122A1022C5827002158314C58222B0
:102A1000E5822BF582E5833AF58322C3E5829BF5B7
:102A200082E5839AF583227C007D00C2007910ED57
:102A30002DFDEC3CFC5002D200EB33FBEA33FA50A4
:102A40000CED2582FDEC3583FC5002D200D9E08CE0
:102A5000838D82A20022C37C007D007910E5823341
:102A6000F582E58333F583ED3DFDEC3CFCED9BFD0C
:102A7000EC9AFC5006ED2BFDEC3AFCB3D9DFE58275
:102A80003582F582E5833583F583EC4D6002D322F0
:102A9000C322C082C3E5829BF582E5839A4582D03A
:102AA0008222C0E0E82582F58274003583F583D068
:102AB000E022C083C082122AA2E0D082D08322C04A
:102AC00083C082122AA2F0D082D08322855A8385C5
:102AD0005B822285835A85825B22C083C082122A50
:102AE000CCA3122AD3D082D08322C083C082122AE0
:102AF000CC122A06122AD3D082D08322C083C0826D
:102B0000122ACC122A10122AD3D082D08322C08358
:102B1000C082122ACC122A1B122AD3D082D083223E
:102B2000C083C082122ACC122A92D082D08322C0C3
:102B300083C082122ACC93D082D08322C083C082E9
:102B4000122ACC122AB2D082D08322C083C0821231
:102B50002ACC122ABFD082D08322E5822BD4F582E0
:102B6000E5833AD4F58322C3E5829B1229B9F58225
:102B7000E5839A1229B9F583223099FDC299F59916
:102B8000C0E074801470FDD0E022122C2DEA122BCC
:102B900079EB122B7922CF2FCF122B8A22E58312C9
:102BA0002B8AE582122B8A22E493B40002A322B47A
:102BB0000D05122BC5A322122B79A380EB742012D2
:102BC0002B79DAF922740D122B79740A122B7922DF
:102BD0007420122B79223098FDC298E59922122B8D
:102BE000D6FA122BD6FB122C4A22122BDECF2FCF75
:102BF00022122BDEF583122BDEF582228587F0B4BC
:102C00001907758DFDD2F78020B49607758DFDC22A
:102C1000F78016B44805758DFA800EB42405758DBD
:102C2000F48006B41206758DE885F08722C0E0C4F2
:102C3000122C3BFAD0E0122C3BFB22540FB40A00BA
:102C400050034430229409444022EA122C56C4FA1C
:102C5000EB122C564A22B4410040022409540F22A0
:102C6000E4F9FAFB7C10E58233F582E58333F583E2
:102C70007D037803E635E0D4F618DDF8DCE8227C45
:102C8000107D037801C3E613C0D030E703C394304E
:102C900030E303C39403F608D0D0DDEAE58313F5EF
:102CA00083E58213F582DCD922B46100500122B49D
:082CB0007B00400122941F2269
:00000001FF
